:10000000AFC0C9C0C8C04EC3C6C0C5C0C4C08AC185
:10001000C2C0C1C0C0C0BFC0BEC02BC3BCC0BBC07B
:10002000BAC0B9C0B8C0B7C0B6C03E20000D0A0003
:100030004F4B0D0A00496E76616C696420656E74E1
:1000400072790D0A004E49584945544143482049A8
:100050004920436F6D6D616E642D4C696E6520495A
:100060006E746572666163650D0A4A756C2032397B
:1000700020323031372031323A33373A31330D0ABA
:1000800000382063796C696E646572730D0A0036FE
:100090002063796C696E646572730D0A00342063A5
:1000A000796C696E646572730D0A0052504D3A2086
:1000B000002C206477656C6C3A2000206465672E04
:1000C0000D0A002D2D2D004C6F6767696E67207338
:1000D0007461727465640D0A004C6F6767696E67BE
:1000E0002073746F707065640D0A00446973706CDE
:1000F0006179206973206F6E0D0A00446973706C1A
:100100006179206973206F66660D0A00556E657807
:1001100070656374656420726573706F6E736520BB
:1001200066726F6D20424C45206D6F64756C650D75
:100130000A005645520043594C0052504D0053544A
:100140004152540053544F500044495350004F4EB5
:10015000004F464600524553455400424C4500006E
:1001600011241FBECFE5D1E0DEBFCDBF10E0A0E679
:10017000B0E0EAE4FFE002C005900D92A436B107BA
:10018000D9F710E0A4E6B0E001C01D92A53AB1078E
:10019000E1F702D0D8C634CF8F929F92AF92BF9230
:1001A000CF92DF92EF92FF920F931F93DF93CF9343
:1001B000CDB7DEB7E2970FB6F894DEBF0FBECDBF66
:1001C00089D042D24DD29DD29BD37894BAD332D427
:1001D000CC24DD2400E010E04E010894811C911C29
:1001E0008AE1A82EB12CAC0EBD1E02C000E010E0CA
:1001F000909189008091A3009817E1F08091890087
:10020000E82FF0E0E556FF4FF0808F5F8093890084
:1002100080918900877080938900A6D0813021F475
:1002200080E061E0B1D006C08C2D6F2DA40121E0EB
:10023000E4D1C82E90918A0080918700981771F0C0
:10024000E92FF0E0E557FF4F60819F5F9F7090932B
:100250008A008D2DA50122E0D0D1D82E8091A40056
:100260008823A1F01092A40082E09AE060E670E09A
:1002700056D554D3882309F4BED376D0882331F0E1
:100280008E2DE39480FF02C06FD0A1D080918800B2
:10029000813079F0813008F4ABCF8230B9F410921C
:1002A0008800012B09F0A2CFF89404B515B5789415
:1002B0009FCF109288000115110509F499CFF89489
:1002C00064B575B57894C80129D290CF1092880092
:1002D000F1D28CCF12B883E389B98AB188698AB91F
:1002E00083B1866083B908955D9BFECF8CB9089574
:1002F00020E004C05D9BFECF2F5FECB9FC01E20F54
:10030000F11DE081EE23B1F7089520E004C05D9B6C
:10031000FECF2F5F3CB9FC01E20FF11D3491332376
:10032000B1F708951F920F920FB60F9211248F9379
:100330009F93EF93FF938091A3009CB1EBE9F0E0D2
:10034000E80FF11D90838F5F8093A3008091A3003D
:1003500087708093A300FF91EF919F918F910F90F1
:100360000FBE0F901F9018958091640008959C0116
:10037000613019F0623039F402C0C7DF089581E0BE
:100380009AE0B9013ED408951F93162F809364001C
:10039000882331F0833060F487EC90E0E8DF08C018
:1003A00089ED90E0E4DF113019F48AE290E0ADDFEE
:1003B0001F9108959C01613019F0623039F402C038
:1003C00097DF089581E09AE0B901A9D40895FF92DA
:1003D0000F931F93DF93CF93CDB7DEB728970FB658
:1003E000F894DEBF0FBECDBFF82E8BEA90E06F2DE4
:1003F000BEDF72D28E010F5F1F4F892B31F06CD29E
:10040000B8014AE050E067D504C0C80163EC70E071
:1004100013D58E010F5F1F4FC8016F2DCBDF81EB0E
:1004200090E06F2DA4DF64D2882339F061D290E090
:10043000B8014AE050E04FD504C0C80163EC70E059
:10044000FBD4CE0101966F2DB5DF8BEB90E06F2DC5
:100450008EDF28960FB6F894DEBF0FBECDBFCF91CA
:10046000DF911F910F91FF9008951F93CF93DF931A
:10047000162F61E670E0F0D4EC01113019F48DE232
:1004800090E043DF209709F4AFC0CE0110D562E3BE
:1004900071E0C9D4892B19F485E490E0A3C0CE01A2
:1004A00006D566E371E0BFD4892BB1F480B390E048
:1004B000807390708032910561F08033910531F046
:1004C000409709F08DC081E890E08CC08FE890E003
:1004D00089C08DE990E086C0CE01E9D46AE371E07D
:1004E000A2D4892BF9F480E090E061E670E0B4D406
:1004F000EC01009719F4812F6ADF76C0D8D46EE33F
:1005000071E091D4892B11F4812F09C0CE01CFD491
:1005100064E471E088D4892B09F062C080E0612F27
:1005200033DF67C0CE01C3D469E471E07CD4892B8A
:1005300091F580E090E061E670E08ED4EC010097E8
:1005400019F4C19913C007C0B2D46EE471E06BD442
:10055000892B21F4E9D18BEE90E044C0CE01A7D4E1
:1005600061E571E060D4892B21F4E0D18BEF90E05C
:1005700039C0CE019CD465E571E055D4892B19F4BE
:1005800080E0CFD105C081E0CCD1CE012FD4DED127
:1005900080E390E027C0CE018AD46BE571E043D4BC
:1005A000892BF1F4123031F481E09AE065E370E0D8
:1005B00028D31FC080E090E061E670E04DD4EC01EC
:1005C00076D465E571E02FD4892B29F433D280E30A
:1005D00090E09BDE0BC080E09AE0BE01A0D306C095
:1005E00085E390E0612FC3DE113019F48AE290E0D8
:1005F0008CDEDF91CF911F9108951F93182FDA01A0
:100600006D3021F06F3759F06A3089F4FD01E10F48
:10061000F11D1082CD01622F28DF10E012C0882367
:1006200081F0213011F48FE75FDE11500AC088316C
:1006300040F4A80FB11D6C93213011F4862F54DEC5
:100640001F5F812F1F91089580B7826080BF83B79D
:10065000856083BF89B7816089BF8CE986BF0895B3
:100660008EB582608EBD89B7886089BF1092880080
:1006700008951F920F920FB60F9211248F938091BD
:100680006500893120F48F5F8093650005C010926A
:10069000650081E08093A4008F910F900FBE0F90B2
:1006A0001F9018951F920F920FB60F9211248F93DF
:1006B0009F931DBC1CBC0EB406FE0AC008B607FE04
:1006C00005C088B7806888BF81E80BC081E009C099
:1006D00008B607FE05C088B7806888BF82E801C0F9
:1006E00082E0809388008EB590E489278EBD88B71C
:1006F000886088BF9F918F910F900FBE0F901F90C1
:10070000189588B3816288BB88B38E6188BB87B334
:100710008E6D87BB82B38C6382BB08956F927F928C
:100720008F929F92AF92BF92CF92DF92FF920F93E0
:100730001F93CF93DF935C01CC24DD243B018824FD
:1007400099246A0C7B1C8C1C9D1C80B3282F30E0E4
:100750002073307020323105D1F12033310509F199
:100760002031310541F060E070E080E090E0AA24A3
:10077000BB24650141C0C601B5012DE230E040E077
:1007800050E0F9D25B016C0184E290E9A0E0B0E0B6
:10079000A80EB91ECA1EDB1E60E873EC89EC91E05E
:1007A0002BC0C601B5012CE330E040E050E0E3D2BD
:1007B0005B016C0180E390ECA0E0B0E0A80EB91EF4
:1007C000CA1EDB1E60E07AE582E692E015C0C60133
:1007D000B5012AE530E040E050E0CDD25B016C018C
:1007E00088E490E2A1E0B0E0A80EB91ECA1EDB1EAC
:1007F00060E077E883E993E0F09081000F2D10E04E
:10080000000F111F0A591F4FA4019301CDD2D80127
:100810002D933C93F394B7E0FB22F0928100F0908B
:1008200082000F2D10E008581F4FC601B501A4012A
:100830009301BAD2F8012083F394F7E0FF22F092FB
:100840008200E6E6F0E0C8E7D0E020E030E040E0FB
:1008500050E060E070E081919191A0E0B0E0280F5D
:10086000391F4A1F5B1F8991680F711D80E0E637B1
:10087000F80789F793E056954795379527959A9508
:10088000D1F7309377002093760083E076956795D3
:100890008A95E1F760938000DF91CF911F910F91CE
:1008A000FF90DF90CF90BF90AF909F908F907F9000
:1008B0006F900895E6E6F0E0A8E7B0E0119211929B
:1008C0001D9280E0E637F807C9F710927700109282
:1008D000760010928000089508B607FE03C020E05D
:1008E00030E004C02091760030917700C90108956E
:1008F00008B607FE02C080E0089580918000089548
:100900008DB188618DB908958FB9769A03C08DB184
:1009100083608DB9769BFBCF8FB108958091840061
:100920000895809384000895C1980895C19A089508
:100930001F93162FC498E8DF812FE6DFC49A1F911A
:1009400008958FEF6FEFF4DFC19808950F931F9311
:10095000DF93CF93CDB7DEB728970FB6F894DEBFFD
:100960000FBECDBF8E010F5F1F4FB8014AE050E0B0
:10097000B2D2F80101900020E9F73197E01BF10BAA
:10098000E130F10579F0E130F10548F0E230F105B0
:1009900061F099812A813B813397B9F40EC08FEFC2
:1009A0006FEF1DC06981605406C06A816053898100
:1009B0008295807F680F8FEF12C0892F8054632F3C
:1009C00060532295207F620F0AC0822F8053929538
:1009D000907F890F6C8160533295307F630FA8DF61
:1009E00028960FB6F894DEBF0FBECDBFCF91DF9132
:1009F0001F910F91089570DF892B41F0829902C0F9
:100A00006BDF02C075DF90E0A1DF08958091830065
:100A10008F5F837080938300880F880F6FE070E092
:100A200002C0660F771F8A95E2F760957095872F51
:100A30007FDF0895C29880E49CE90197F1F7C29A9C
:100A400088EE93E020E931E0F9013197F1F7019761
:100A5000D9F708956F927F928F929F92AF92BF9233
:100A6000CF92DF92EF92FF920F931F93CF93DF937A
:100A70005C016B0194EA892E91E0992E88EC682E36
:100A8000712C04C0C39AC3010197F1F7C398C40144
:100A90000197F1F78FEF38DFF5018083F501808151
:100AA0008E5F823078F38FEF2FDF082F10E0F60192
:100AB000118300838FEF28DFF82EEE240E0D1F1D0B
:100AC000F601118300838FEF1FDF182F00E0C82F7E
:100AD000D0E0CF771DC08FEF17DF282FF601808180
:100AE0009181FAE080309F0721F082509A4079F49A
:100AF00003C0822FF9DB0BC080918700E82FF0E064
:100B0000E557FF4F20838F5F8F70809387000F5FC3
:100B1000802F90E08C179D07F4F2C39A17FDB6CF93
:100B2000DF91CF911F910F91FF90EF90DF90CF90C9
:100B3000BF90AF909F908F907F906F9008956F922D
:100B40007F928F929F92AF92BF92CF92DF92EF925D
:100B5000FF920F931F93CF93DF93682E762EC72EAD
:100B60007A01CA0170D1082FDD2434EAA32E31E0C6
:100B7000B32E28EC822E912C04C0C39AC401019795
:100B8000F1F7C398C5010197F1F7862DBDDE8E3FC1
:100B9000A1F3872DB9DE8C2DB7DECD2DD0E001314C
:100BA00080F080E9B1DECE0DDF1D10E0FE01849102
:100BB000ABDE1F5F21961031C9F70051F0E1DF0E67
:100BC0000EC0802FA1DECE0DDF1D10E005C0FE019E
:100BD00084919ADE1F5F21961017C8F300E0C39A34
:100BE000002379F6DF91CF911F910F91FF90EF9045
:100BF000DF90CF90BF90AF909F908F907F906F903D
:100C000008950F931F93DF93CF9300D00F92CDB72A
:100C1000DEB78C01AB0180E1B80191DF8399FECF93
:100C2000CE010196BE016E5F7F4F14DF8981803255
:100C300011F020E009C020E08A819B818017910794
:100C400009F021E081E02827822F0F900F900F906C
:100C5000CF91DF911F910F9108956F927F928F92A4
:100C60009F92AF92BF92CF92DF92EF92FF920F933B
:100C70001F93CF93DF93682E762EC72E7A01FA0149
:100C800001900020E9F731970E2F041BDD2454EA70
:100C9000A52E51E0B52E48EC842E912C04C0C39AA9
:100CA000C4010197F1F7C398C5010197F1F7862DAB
:100CB0002BDE8E3FA1F3872D27DE8C2D25DECD2D5B
:100CC000D0E0013170F080E91FDECE0DDF1D10E0B5
:100CD00089911ADE1F5F1031D9F7005180E1D80EDB
:100CE0000CC0802F11DECE0DDF1D10E003C08991F6
:100CF0000BDE1F5F1017D8F300E0C39A002399F6AC
:100D0000DF91CF911F910F91FF90EF90DF90CF90E7
:100D1000BF90AF909F908F907F906F9008950F93AA
:100D20001F93DF93CF9300D00F92CDB7DEB78C0126
:100D3000AB0180E1B80191DF8399FECFCE0101962E
:100D4000BE016E5F7F4F86DE8981803211F020E028
:100D500009C020E08A819B818017910709F021E07A
:100D600081E02827822F0F900F900F90CF91DF9175
:100D70001F910F910895FF27EE27BB27AA2760FF39
:100D800004C0A20FB31FE41FF51F220F331F441F1F
:100D9000551F969587957795679589F700977607FC
:100DA00071F7CF01BD010895A1E21A2EAA1BBB1B4A
:100DB000FD010DC0AA1FBB1FEE1FFF1FA217B30727
:100DC000E407F50720F0A21BB30BE40BF50B661F3D
:100DD000771F881F991F1A9469F760957095809501
:100DE00090959B01AC01BD01CF010895FC018827BE
:100DF0009927E89421912032E9F3293010F02E3020
:100E0000C8F32B3239F02D3231F4689403C059D035
:100E1000820F911D219120532A30C8F31EF4909522
:100E200081959F4F0895FB01DC018D9105908019FC
:100E30000110D9F3990B0895FB01DC0105900D9287
:100E40000020E1F70895FC0105900020E9F7809566
:100E500090958E0F9F1F089545E850E001D00895AA
:100E6000FA01A191B081009719F41097E1F0CD013A
:100E7000DC01CD010D90002011F4C00113C0FB0175
:100E80002191222319F02015D9F7F3CFFB012191ED
:100E9000201519F41E92119606C02223C1F70D9059
:100EA0000020A1F7D001FA01A193B0830895DC01DD
:100EB0006C9161566A3108F0605E6F5B6D93C1F7AB
:100EC0000895BC01880F991F880F991F860F971FDF
:100ED000880F991F0895FB019F0142306CF0453245
:100EE0005CF4642F77271BD0805D8A330CF0895D1A
:100EF0008193CB010097A9F71082C90100C0DC01E2
:100F0000FC01672F71917723E1F7329704C07C9140
:100F10006D9370836291AE17BF07C8F30895AA1B43
:100F2000BB1B51E107C0AA1FBB1FA617B70710F0D4
:100F3000A61BB70B881F991F5A95A9F78095909506
:0A0F4000BC01CD010895F894FFCF25
:040F4A000020000083
:00000001FF
